:1000000012C01895189518951895189506C3189547
:100010001895189518951895189518951895189578
:100020001895189518958FE58DBFC0EEE8EF4E2E08
:1000300084E08EBFD3E0F2E05F2EEEEFF3E0A0E6C7
:10004000B0E088278D933197E9F766248FEF87BB5F
:10005000BC988FEF84BB8FEF81BBBC98C49A11D43E
:10006000789483E080936F0084E08093700087E051
:100070008093710088E08093720086E08093730023
:1000800080E08093740082E08093750089E0809323
:10009000760085E08093770081E0809378008AE0A5
:1000A000809379008AE080937A008AE080937B00D5
:1000B0008AE080937C008AE080937D008AE08093D0
:1000C0007E0081E080937F0000917F000E3410F06D
:1000D00009F01AC08AE090E0DAD1409190000091D6
:1000E000A900041709F401C00FC0409183000091DA
:1000F000AA00041709F401C007C0AFE7B0E08C9173
:100100008F5F8C9308F4E0CF8CED90E0C0D18091AC
:1001100090008093A900809183008093AA00E0E979
:10012000F0E040D2A7E6B0E00D931D932D933D93F0
:10013000E7E6F0E0A4E6B0E056D2009165004AE0C0
:10014000F1D3AEE6B0E00C9300916E004AE0049F5C
:10015000ADE6B0E00C920091650040916D00041B8B
:10016000AEE6B0E00C93009165004AE0DBD3ADE66B
:10017000B0E00C93009166004AE0D4D3ACE6B0E066
:100180000C9300916C004AE0049FABE6B0E00C9247
:100190000091660040916B00041BACE6B0E00C934C
:1001A000009166004AE0BED3ABE6B0E00C93ABE64C
:1001B000B0E0AD90BB24AFE6B0E0AA0DBB1D8C91C2
:1001C00080936B00ACE6B0E0AD90BB24AFE6B0E04E
:1001D000AA0DBB1D8C9180936C00ADE6B0E0AD9094
:1001E000BB24AFE6B0E0AA0DBB1D8C9180936D00DF
:1001F000AEE6B0E0AD90BB24AFE6B0E0AA0DBB1D0B
:100200008C9180936E0000E110E020E030E0ACE6DD
:10021000B0E04C9155276627772749D3A0E6B0E098
:100220000D931D932D933D93A0E6B0E00D911D918C
:100230002D913C91ADE6B0E04C915527662777278C
:100240006CD3A0E6B0E00D931D932D933D93A0E6F3
:10025000B0E08C9182BB85B3A0E6B0E08D93882797
:100260008D938D938C93A0E6B0E00D911D912D910F
:100270003C9140EF50E060E070E0FBD0A0E6B0E0E1
:100280000D931D932D933D93A0E6B0E00D911D912C
:100290002D913C91AEE6B0E04C915527662777272B
:1002A0003CD3A0E6B0E00D931D932D933D93A0E6C3
:1002B000B0E08C9185BB88B3082F11272227332704
:1002C00040EF50E060E070E0D4D0A0E6B0E00D93E5
:1002D0001D932D933D93A0E6B0E00D911D912D91BE
:1002E0003C91ABE6B0E04C9155276627772715D3B4
:1002F000A0E6B0E00D931D932D933D93A0E6B0E0F2
:100300008C9188BB009183000D3210F009F001C080
:1003100005C080918D008F7780938D00D2CE000034
:100320000895F894FFCF03000400070008000600BA
:1003300000000200090005000100000000000000AC
:1003400000000000000008D0A8D200FC10D00895E2
:1003500003D01ED001F8F9CF0024E89457FF02C063
:1003600009D0689400F80BD010F80124089502D049
:1003700009D00895509540954F5F5F4F0895E894D8
:1003800017FF0895009510950F5F1F4F689408950B
:10039000352F242FE894452B11F468940895512F9C
:1003A000402F0027112780E1440F551F001F111F08
:1003B000021B130B416018F4020F131F4E7F8A9526
:1003C00099F7089500FC05D0089530D005D001F8C4
:1003D000F9CF37D03FD00895842F952FA62FB72F70
:1003E000E894452B462B472B11F468940895402F31
:1003F000512F622F732F0027112722273327F0E276
:10040000440F551F661F771F001F111F221F331F28
:10041000081B190B2A0B3B0B416028F4080F191F0E
:100420002A1F3B1F4E7FFA9559F708950024E89440
:1004300077FF02C006D0689400F809D010F80124B4
:10044000089512D04F5F5F4F6F4F7F4F0895E8942C
:1004500037FF089500951095209530950F5F1F4F39
:100460002F4F3F4F68940895409550956095709533
:100470000895042315232623372308953197F1F790
:100480000895689462F80895E89462F80895EF93E7
:10049000FF93EE27E82BE92B31F0E8EEF3E03197FC
:1004A000F1F70197D1F7FF91EF91089589B78F7E0A
:1004B00089BF80E08FBD8AE08EBD80E090E09093A0
:1004C0004D0080934C0084ED90E390934B0080931B
:1004D0004A0088B7806188BF89B7806189BF089565
:1004E00093E0ADE002C096E0AAE0B0E08FB7F894E8
:1004F00001910D939A95E1F78FBF0895F1DF0E2DCD
:100500000A95802F0295003220F01F2D137009F4F8
:100510000395DA940D0D11279927EAE2F5E0A8E199
:10052000BB27F8D1080F111F0895000F1B2A384769
:1005300055647381909ED4DF0F2D11274CE355270E
:1005400002DF55270E0D151F4CE3222733276627A0
:100550007727ADD10D0D131F231F0895C1DFDF9243
:10056000EF92FF920F2D1127222733274DE651E0FE
:1005700060E070E09CD1FF904F2D4D5F4695469511
:10058000552766277727C9D1EF90DF900F931F93E8
:100590002F933F93B4DF222733277F916F915F9191
:1005A0004F91BBC1A0DFAF92BF92CF92D8DF40E89E
:1005B00051E561E070E07BD1FF90EF90DF900F9309
:1005C0001F932F933F93B8DF7F916F915F914F916E
:1005D000A4C1019111912191308140E851E561E080
:1005E00070E0F3DE0DC0AF93BF93F3DFBF91AF9127
:1005F000DD92ED92FD92089501911191219130814A
:1006000040E15EE060E070E0E0DEF42E4CE350E0BC
:100610009FDEE42ED02E08950895FF93EF936F93FD
:100620008F939F937F938FB78F93E2E8F0E063857A
:1006300064FD40C070817395708386B366FF02C00D
:1006400090E1892784FB80F9862780FF33C060F919
:100650008827808356F0E89470938000763008F005
:10066000689435D08287718725C070938100763376
:10067000C8F09927918362FF1DC095879687828174
:1006800087878381808B8481818B8581828B868122
:10069000838B8781848760686B7F638763FDEBD082
:1006A000A7D00CC0918193959B3311F4808586FF70
:1006B0006B7F91835ED063870EF4D2D08F918FBF12
:1006C0007F919F918F916F91EF91FF911895718517
:1006D0008285918116F473957D7F869587F982874F
:1006E000943129F4808777270EF0706808959C3143
:1006F00019F430D0828338C0933219F429D083831F
:1007000033C0993219F423D0848308959C3229F49C
:1007100082958695877087830895913319F416D052
:1007200085830895993319F416D0868308959A33F2
:1007300061F41AD051F486A183958C3309F488278B
:10074000928196A3891709F4646008958695869529
:100750008F7786958F7784FD865085FD8C5086FD3A
:10076000885187FD8053089570FB769577F9707FE7
:100770000895E894858583958587883208F40895DF
:10078000882785878685839586878C3388F17727A8
:1007900076878785839587878C3350F17787808923
:1007A0008395808B883120F1708B81898395818B33
:1007B0008D31F0F092898F3111F080F408C09430BF
:1007C00069F0963059F0993049F09B3039F0923009
:1007D00079F47389737011F48E3150F071E0718B7C
:1007E0009395928B9D3020F0728B83898395838BB8
:1007F0000F921F922F923F924F925F927F92AF92F1
:10080000BF920F931F932F933F934F935F936F93D9
:100810007F938F939F93AF93BF93CF93DF93EF9388
:10082000FF938FB78F937BDD8F918FBFFF91EF91F8
:10083000DF91CF91BF91AF919F918F917F916F91F8
:100840005F914F913F912F911F910F91BF90AF906A
:100850007F905F904F903F902F901F900F90089542
:10086000E2E8F0E063856F7E6387BF93AF931EDE9F
:10087000AF91BF910895E2E8F0E06385606163871E
:100880000895882780938D00EBCF70918A00882788
:1008900075FB80F974FB81F908950F92B801469FAA
:1008A0008001479F100D569F100D0F9008950F92D5
:1008B0001F922F92C801D901489F80014A9F900141
:1008C0004B9F202C499F100D211D321D5A9F202C1B
:1008D000589F100D211D321D599F200D311D689FFD
:1008E000200D311D699F300D789F300D2F901F9086
:1008F0000F900895C89531960020089591E005C0A5
:1009000092E003C094E001C098E0F4DF0D929A9564
:10091000E1F70895E80FF91FF1CF040F151F261F07
:10092000371F0895FF93881BF9E0001FFA9511F413
:10093000FF910895881F841B18F4840F8894F5CFC5
:040940000894F3CF55
:00000001FF
